:03000000020300F8
:05001B00C28EC28B3211
:0C010000758D3C758BAFD28E208EFD22D9
:10020000D2B77928120100D9FBE49360229430AA76
:1002100083AB8290036393F590D297790412010027
:10022000D9FBC2978A838B82A3120100020209794B
:1002300064120100D9FBD2B679C812010012010084
:10024000B2B6D9F6C2B6C2B77928120100D9FB22DC
:10030000C2B7C2B6758911C28CC28ED2ABD2AFC28F
:100310009730B00690033712020030B106900342C6
:1003200012020030B20690034D12020030B3069064
:10033000035812020080FE303637373737373737E9
:1003400037003036383838383838383800303136B9
:100350003636363636363600303138383838383872
:0E036000383800576E5E3E6D5D3D6B5B3B00B6
:00000001FF
